:10000000ADC1C4C1C3C1C2C1C1C1C0C1BFC1BEC1F4
:10001000BDC1BCC1BBC1BAC1B9C1B8C1556E697659
:10002000657273616C20524620506F7765726D6502
:1000300074657220202020444C354E4547202020F6
:100040000A004144432D72617776616C75652041E9
:100050004443312020414443322020242D2D2D20A3
:1000600020242D2D2D200A0044696F646520202056
:10007000202D2D2D203A78782E78782064422D205E
:100080006175746F202020204144432D0A004C6F7D
:1000900067416D702020202D2D2D203A78782E7804
:1000A000782064422D2066203D202D2D3030204DBB
:1000B000487A0A00546865726D6F2020202D2D2D1E
:1000C000203A78782E78782064422D207A65726FF5
:1000D0002D61646A3A202D2D0A002020426174743B
:1000E000657279202020202D2E2D20566F6C747380
:1000F00020205374617475733A202D6F6F2D0A00A0
:1001000020205741524E494E4720202020204F5654
:1001100045524C4F414420207265647563652070E0
:100120006F7765720A000F00110015001A001F009A
:1001300025002C0033003C004600530060006E0098
:1001400080009300AB00C400E000FE0021014C01E0
:100150007901AC01E90128027602C8022203870373
:10016000FFFF0A000C000F00110015001A0020000C
:10017000270030003C0049005B006F008800A500AC
:10018000C800F50026016001A701F5015602C00272
:100190003903C803FFFF27002A002D003100340077
:1001A000380041004B0055005F0069008500A20047
:1001B000BF00EC0019016601B3010102940227039C
:1001C000F203FFFFA100A300A600AA00AD00B1004A
:1001D000B600BB00C000C600CC00D100D700DD00D7
:1001E000E300E900EF00F500FB00020108010E0149
:1001F00015011B01220129012F0135013C0142019A
:1002000049014E0155015B01620168016E017401F3
:100210007A01810187018D0193019901A001A60155
:10022000AC01B201B801BF01C501CA01D001D701BB
:10023000DD01E301E901EF01F501FB010102060225
:100240000B020F02140217021B02FFFFAA00AE00EE
:10025000B200B600BB00C000C600CB00D100D70082
:10026000DD00E200E800EE00F400F9000001050105
:100270000B01100116011C01220127012C01320182
:1002800038013D01430148014E01530158015E010F
:10029000630169016F0175017A01800185018B019C
:1002A000910197019C01A201A801AE01B401B9011D
:1002B000BF01C501CB01D001D601DC01E201E8019B
:1002C000EE01F401F901000205020A020F02130215
:1002D0001702FFFFA600A900AD00B200B600BC00E7
:1002E000C200C800CE00D500DC00E200E900F0004A
:1002F000F700FE0006010D0114011B0122012A0175
:10030000310138013F0145014D0153015A0161019D
:1003100067016D0174017B01810188018F019501E5
:100320009C01A201A901B001B701BD01C401CA012C
:10033000D101D801DE01E501EB01F101F701FD0179
:1003400003020902100217021D0224022A023002CF
:10035000340238023A023C023F02FFFF11241FBE62
:1003600020E0A89521BD20E025BFEAE9FDE0A0E658
:10037000B0E003C0C89531960D92A636D9F7A6E62F
:10038000B0E001C01D92AD38E9F702C000C0189579
:10039000CFEDD0E0DEBFCDBF8FEF81BB81E384BB6B
:1003A00082E087BB87E388BB43D481E079D165D401
:1003B0008FEF54D18FEF52D183E08093600070D1E2
:1003C0005CD4C6B3C0FF10C13C2F3071C4FFD4C091
:1003D0009C2F9470C2FFC4C0809160009927843024
:1003E000910521F481E014D16CD2EACF85309105DA
:1003F0000CF457C085309105F9F481E009D1D92F6B
:10040000C82F5FD2C032D10581F0A19738F48CE3B8
:1004100080938A008DE280938B00D2CF8DE280930F
:100420008A008EE380938B00CBCF8FE680938A0087
:100430008BE680938B00C4CF069709F0C1CF83E091
:10044000E7D0D92FC82F82E0C935D80728F184E634
:1004500080938B0087E68093880083E0D695C795CC
:100460008A95E1F780E090E020E00A962F5FC817B8
:10047000D907D8F72150C81BD90B8C2F9D2F0A966E
:10048000982F2A302CF02A5081E380937400B8C052
:1004900080E280937400B4C082E780938B0080E791
:1004A000DACF82309105D9F581E0B2D0D92FC82FAB
:1004B0008C2F8F70E9D08093840044E0D695C79547
:1004C0004A95E1F78C2F8F70DFD08093830034E062
:1004D000D695C7953A95E1F78C2F8F70D5D080933C
:1004E000820082E095D0D92FC82F8C2F8F70CCD06E
:1004F00080938A0024E0D695C7952A95E1F78C2F42
:100500008F70C2D08093890094E0D695C7959A9554
:10051000E1F78C2F8F70B8D08093880051CF03976C
:1005200009F04ECF8091610073D0D92FC82F8091F0
:100530006200882389F0C333D10518F482E08093E8
:100540006100C95CD34018F081E080936100809124
:1005500061005ED0D92FC82F8C2F9D2FB2D130CF04
:1005600080916400882321F09093640046D134CFB9
:1005700081E080936400FACF80916000833081F045
:1005800080916000843011F038D122CF80916300D7
:100590008F5F809363008330B8F310926300F4CFD1
:1005A00080916200882311F03093610020916100F6
:1005B000822F99278130910599F08230910544F47A
:1005C000892BF1F63093620081E080936100D8CFEF
:1005D0000297B1F63093610081E080936200D0CF42
:1005E0002F5F20936100CCCF809160008F5F80935C
:1005F0006000873018F082E080936000FED0E4CE87
:10060000205D20937500905D90937700D9CEFFCF49
:100610001F93CF93DF93982F86EE86B997B9C0E0EA
:10062000D0E010E084E0ECD2181768F481E016D036
:1006300024B185B19927982F8827820F911DC80F63
:10064000D91F1F5FEFCF54E0D695C7955A95E1F7B4
:100650008C2F9D2FDF91CF911F9108950F931F93A2
:10066000082F1DBC1CBC18B786E0CAD2182B18BFB7
:1006700083E08EBD0BBD1ABC18B786E0C1D218232B
:10068000D9F31F910F910895805D8A3308F0895F37
:1006900099270895843209F482E0805899270895B3
:1006A0008F929F92AF92BF92CF92DF92EF92FF9282
:1006B0000F931F93CF93DF93A82EBB2420E030E04D
:1006C000E0E0CE2EE1E0DE2E7AEDE72E70E0F72EB0
:1006D00004EB10E0CEE8D0E0A8E6B0E062E470E021
:1006E0004CE150E08A2D99278430910509F456C0D9
:1006F0008530910554F582309105E1F08330910504
:1007000074F4019709F057C0822E932E88E690E08A
:10071000880E991EF52FE42FC895802D49C0822E92
:10072000932E88E690E0880E991EFB2FEA2FC8953D
:10073000802D3EC0822E932E88E690E0880E991E72
:10074000F72FE62FC895802D33C086309105D9F05C
:10075000863091056CF0079771F5822E932E88E60E
:1007600090E0880E991EFD2DEC2DC895802D20C09F
:10077000822E932E88E690E0880E991EF12FE02FAE
:10078000C895802D15C0822E932E88E690E0880EA5
:10079000991EFF2DEE2DC895802D0AC0822E932E16
:1007A00088E690E0880E991EFD2FEC2FC895802DCD
:1007B000F92DE82D80830894C11CD11C0894E11CFC
:1007C000F11C0F5F1F4F219611966F5F7F4F4F5F98
:1007D0005F4F2F5F3F4FB394F3E2FB1508F082CFDA
:1007E000DF91CF911F910F91FF90EF90DF90CF900D
:1007F000BF90AF909F908F9008958091600050DFE0
:100800003CD284E62BDF0895282F392F8091640095
:100810008130F1F130936700209366008BE2809382
:100820007500332374F180E090E060E02817390709
:1008300034F088519C4F6F5F28173907D4F7615007
:10084000281B390B28513C4F80E090E040E02817EE
:10085000390734F08C599F4F4F5F28173907D4F769
:100860004150281B390B2C593F4F80E090E050E05D
:1008700028173907A4F00A965F5F28173907DCF7B5
:100880000EC08DE280937500309521953F4FCBCF00
:100890008091660090916700281B390BBFCF281B01
:1008A000390B932F822F0A96605D60937600405D2E
:1008B00040937700515D50937900805D80937A007A
:1008C0000895BF92CF92DF92EF92FF920F931F9302
:1008D000CF93DF93E82EF92E80916000E1DE2BD1DB
:1008E00080916000833009F4CFC080916000843033
:1008F00009F456C080916000853091F1BB2031F140
:100900008FEF0F3F1807F9F00C1B1D0BEC1AFD0AB7
:10091000E4E6F0E09F2D8E2D6E2F7F2F03D2712FF6
:10092000602F12D2262F372FCB0CD11C9D2D8C2D52
:100930006E2F7F2FF7D1280F391F24563040932F69
:10094000822F62DFEEC087E0ABDEEBC08CE38093EA
:1009500074009D2D8C2D64E670E0E4D155DFE1C07C
:10096000BB24CB2DDD27CC0FDD1F0C2F1D2F0A56EE
:100970001E4F912F802F4ED1E816F90678F4CC2423
:10098000DD24912F802F46D1082F192FCC56DE4F12
:100990008C2F9D2F3FD1D92FC82FB0CFB394E1CF4B
:1009A00080916300882309F44DC0809163008130F9
:1009B00039F180916300823009F09CCFBB24CB2DAC
:1009C000DD27CC0FDD1F0C2F1D2F0C521D4F912F3B
:1009D000802F20D1E816F90688F4F4ECCF2EFFEF33
:1009E000DF2E912F802F16D1082F192FCE52DD4FD9
:1009F0008C2F9D2F0FD1D92FC82F7CCFB394DFCF51
:100A0000BB24CB2DDD27CC0FDD1F0C2F1D2F045B4E
:100A10001D4F912F802FFED0E816F90688F4A4EC24
:100A2000CA2EAFEFDA2E912F802FF4D0082F192F76
:100A3000C65BDD4F8C2F9D2FEDD0D92FC82FB9CF9E
:100A4000B394DFCFB82ECB2DDD27CC0FDD1F0C2FBD
:100A50001D2F0C531E4F912F802FDCD0E816F90666
:100A600088F4B4ECCB2EBFEFDB2E912F802FD2D0A9
:100A7000082F192FCE53DE4F8C2F9D2FCBD0D92F7F
:100A8000C82F93CFB394DFCF80916100813039F1CB
:100A900080916100823009F028CFBB24CB2DDD2767
:100AA000CC0FDD1F0C2F1D2F0E591E4F912F802FA5
:100AB000B1D0E816F90688F482EEC82E8FEFD82E52
:100AC000912F802FA7D0082F192FC05ADE4F8C2FBF
:100AD0009D2FA0D0D92FC82F08CFB394DFCFBB2430
:100AE000CB2DDD27CC0FDD1F0C2F1D2F0A5D1E4FD8
:100AF000912F802F8FD0E816F90688F492EFC92E37
:100B00009FEFD92E912F802F85D0082F192FCC5DE4
:100B1000DE4F8C2F9D2F7ED0D92FC82FB9CFB39405
:100B2000DFCFDF91CF911F910F91FF90EF90DF907A
:100B3000CF90BF90089580916400882309F454C039
:100B400082E78093710085E6809372008CE6809343
:100B5000730080E280937E0080916000833019F101
:100B600080916000843009F04AC080916300992729
:100B70008130910589F08230910554F4892B09F078
:100B80003EC080E28093840085E38093850037C077
:100B90000297A9F582E301C081E38093840083E397
:100BA000809385002CC080916200882391F081E6BB
:100BB0008093800085E78093810084E780938200A2
:100BC0008FE68093830080916100805D80938B002D
:100BD000C7CF8DE68093800081E6809381008EE60A
:100BE0008093820080E2EDCF81E68093710082E6FF
:100BF0008093720083E7809373008DE6ABCF0895F6
:100C0000282F81E090E002C0880F991F2A95E2F713
:100C100099270895F92FE82F3196C895802D31979F
:100C20009927982F8827C895202D820F911D089508
:100C3000CF938AE013DD85B38F7C85BBC1E080E371
:100C400090E066D081E00ADDCF5FC430C0F388E376
:100C500090E05ED081E002DD8CE090E059D081E050
:100C6000FDDC81E090E054D084E0F8DC82E090E0AC
:100C70004FD084E0F3DCCF9108950F931F93CF936F
:100C800085B38F7D85BB82E890E042D084E0E6DCCE
:100C900085B3806285BBC0E008E610E0F12FE02F4D
:100CA00081910E2F1F2F992733D0CF5FCC30B0F317
:100CB000C1E080E290E02CD0CF5FC530D0F3C8E136
:100CC00000E810E0F12FE02F81910E2F1F2F9927C0
:100CD0001FD0CF5FC432B0F385B38F7D85BB82EC6C
:100CE00090E016D084E0BADC85B3806285BBCCE0AE
:100CF00004E710E0F12FE02F81910E2F1F2F99278D
:100D000007D0CF5FC831B0F3CF911F910F910895F5
:100D100082BB85B3806185BB85B38F7E85BB81E057
:100D20009DDC08955527002480FF02C0060E571F42
:100D3000660F771F6115710521F0969587950097CD
:100D400099F7952F802D089597FB092E07260AD035
:100D500077FD04D00CD006D000201AF47095619570
:100D60007F4F0895F6F7909581959F4F0895AA1BA0
:100D7000BB1B51E107C0AA1FBB1FA617B70710F086
:100D8000A61BB70B881F991F5A95A9F780959095B8
:0A0D9000682F792F8A2F9B2F0895FA
:060D9A0001000100000051
:00000001FF
